:03000000020100FA
:03000B000204A646
:03001B000203C31A
:10010000C290C291C281C28075A7167880E4F6D8E9
:10011000FD75F6044384047F0A75AD28758911D2F4
:100120008ED2AB4392DB438512208702D207208513
:1001300002D2627521247522FA7523247524FA757A
:1001400025247526FA7527247528FAD2AFC292792C
:1001500000719479007194519CC2027C0D75290044
:10016000752A00C28375A61E75A6E1519C3007034F
:100170000202AB3095ED78FF309508740A719BD878
:10018000F780E0B8E60702018FD28380D650D4B85A
:10019000BE0302019740F278FF209508740A719B14
:1001A000D8F780B3B8E6030201AC50F6B8B4030246
:1001B00001B440EE78FF309509D8FB80E5D283008A
:1001C00080E0B8B0030201D8400E7419719B3095DD
:1001D000ECE8C3940AF880DEB850030201DE78FF31
:1001E00020950500D8FA80D5B8D0030201FE400E54
:1001F0007419719B2095C6E8C3940AF880E2B89000
:10020000030202065004D302020BC3E52913F529A9
:10021000E52A13F52ADC9D304F02D2020203452065
:100220004E0AC29020620C9172020233D290206278
:1002300002914C204D05C29102023DD291740030D2
:100240005302D2E0305402D2E1F5347C05C3E529F3
:1002500013F529E52A13F52ADCF3852A3371A1E584
:1002600034C2ABB4000B853521853622D258020248
:1002700095B4010B853523853624D259020295B4F5
:10028000020B853525853626D25A020295853527FB
:10029000853628D25BD2AB91D5020157E5AD20E17E
:1002A00004DF04D2057F0A220201632086FA78FF68
:1002B000208608740A719BD8F780EDB8E603020225
:1002C000C350E5B8BE030202CB40DD78FF3086099B
:1002D000740A719BD8F7020157B8E6030202E15095
:1002E00011B8B4030202E9400978FF208608D8FB60
:1002F00080E4D28380E0B8C0030202FE50F4B8501C
:100300000302030478FF3086060000D8F980E3B8C2
:10031000D003020325400E7419719B3086D4E8C3C4
:10032000940AF880E1B8900302032D5004D302032D
:1003300032C3E52913F529E52A13F52ADCAB304F42
:1003400002D20280007400304E022401304D02249B
:1003500001304C022401304B022401304A022401B6
:100360003049022401304802240130570224013070
:100370005602240130550224013054022401305326
:1003800002240120E00620020602021F2002FA02D7
:1003900001BD790A74FA719BD9FA220000D5E0FBFD
:1003A00022E53375F004A424E8F535F53BE5F03497
:1003B00003F536F53C7400C39535F5357400953674
:1003C000F53622C0D0F52FC28EC297C296C284C223
:1003D00094E530B4000E85218B85228D305838D2BB
:1003E00097020417B4010E85238B85248D3059277D
:1003F000D296020417B4020E85258B85268D305ABD
:1004000016D284020417B4030E85278B85288D30FD
:100410005B05D294020417E5302401F530B40525BC
:10042000753000758BBC758DB7300519E52D24012D
:10043000B41410752D00309205C292020445D29278
:10044000020445F52DD28EE52FD0D032206034D273
:1004500060C280758A06758CFF7537067538FF7522
:100460003906753AFF7A647E28D2A9D28CD2060268
:10047000048330060EC260C2A9C28CC281C206C209
:1004800001D28022C3E5399402F539E53A9400F5AA
:100490003AE5372402F537E5383400F538DA06C294
:1004A000A9C28CD28122C0D0F52FC28C30000CC2E0
:1004B00000C28185378A85388C800AD200D2818536
:1004C000398A853A8CD28C206206DE047E2891849B
:1004D000E52FD0D03230620DE534B40008E533B4F6
:1004E0008D050204E980714057B4EA030204F1402B
:1004F0000E200164C2A9C280C28CD281D2012274B2
:10050000F4C3953BF5317407953CF532C2A97400EC
:10051000C39531F53774009532F53874F4C39531CD
:10052000F53174019532F5327400C39531F53974A3
:10053000009532F53AC280D2A9D28CD20602055675
:10054000C2A9C28CC281C206B46005D2800205561F
:09055000500280F7C280C20122B2
:00000001FF
